 sgx_flip_test

 Timestamp is 4be8c2c3 (Tue May 11 11:36:51 2010)

 Preferred load address is 00010000

 Start         Length     Name                   Class
 0001:00000000 00000004H .CRT$XCA                CODE
 0001:00000004 00000004H .CRT$XCZ                CODE
 0001:00000008 00000004H .CRT$XIA                CODE
 0001:0000000c 00000004H .CRT$XIZ                CODE
 0001:00000010 00000004H .CRT$XPA                CODE
 0001:00000014 00000004H .CRT$XPZ                CODE
 0001:00000018 00000004H .CRT$XTA                CODE
 0001:0000001c 00000004H .CRT$XTZ                CODE
 0001:00000020 00000c38H .rdata                  CODE
 0001:00000c58 0000002aH .rdata$debug            CODE
 0001:00000c84 00001750H .text                   CODE
 0001:000023d4 00000018H .xdata                  CODE
 0001:000023ec 00000028H .idata$2                CODE
 0001:00002414 00000014H .idata$3                CODE
 0001:00002428 000000b0H .idata$4                CODE
 0001:000024d8 0000013cH .idata$6                CODE
 0001:00002614 00000000H .edata                  CODE
 0002:00000000 000000b0H .idata$5                DATA
 0002:000000b0 00000008H .data                   DATA
 0002:000000b8 00000010H .bss                    DATA
 0003:00000000 00000080H .pdata                  DATA

  Address         Publics by Value              Rva+Base       Lib:Object

 0000:00000000       ___safe_se_handler_count   00000000     <absolute>
 0000:00000000       ___safe_se_handler_table   00000000     <absolute>
 0001:00000000       __xc_a                     00011000     corelib0:crt0init.obj
 0001:00000004       __xc_z                     00011004     corelib0:crt0init.obj
 0001:00000008       __xi_a                     00011008     corelib0:crt0init.obj
 0001:0000000c       __xi_z                     0001100c     corelib0:crt0init.obj
 0001:00000010       __xp_a                     00011010     corelib0:crt0init.obj
 0001:00000014       __xp_z                     00011014     corelib0:crt0init.obj
 0001:00000018       __xt_a                     00011018     corelib0:crt0init.obj
 0001:0000001c       __xt_z                     0001101c     corelib0:crt0init.obj
 0001:0000003c       ??_C@_0BD@FOHFKAOE@INVALID?5ERROR?5CODE?$AA@ 0001103c     sgx_flip_test.obj
 0001:00000050       ??_C@_09KMCHPOPM@PVRSRV_OK?$AA@ 00011050     sgx_flip_test.obj
 0001:0000005c       ??_C@_0BF@KHEAJDEG@PVRSRV_ERROR_GENERIC?$AA@ 0001105c     sgx_flip_test.obj
 0001:00000074       ??_C@_0BL@BOENCAIM@PVRSRV_ERROR_OUT_OF_MEMORY?$AA@ 00011074     sgx_flip_test.obj
 0001:00000090       ??_C@_0BN@IHBDMIPO@PVRSRV_ERROR_TOO_FEW_BUFFERS?$AA@ 00011090     sgx_flip_test.obj
 0001:000000b0       ??_C@_0BO@EGNEIFEA@PVRSRV_ERROR_SYMBOL_NOT_FOUND?$AA@ 000110b0     sgx_flip_test.obj
 0001:000000d0       ??_C@_0BL@BKMGFOLH@PVRSRV_ERROR_OUT_OF_HSPACE?$AA@ 000110d0     sgx_flip_test.obj
 0001:000000ec       ??_C@_0BM@LGNAOM@PVRSRV_ERROR_INVALID_PARAMS?$AA@ 000110ec     sgx_flip_test.obj
 0001:00000108       ??_C@_0BN@MGJEIKFE@PVRSRV_ERROR_TILE_MAP_FAILED?$AA@ 00011108     sgx_flip_test.obj
 0001:00000128       ??_C@_0BK@JHPIKHJG@PVRSRV_ERROR_INIT_FAILURE?$AA@ 00011128     sgx_flip_test.obj
 0001:00000144       ??_C@_0CE@POPMCOCG@PVRSRV_ERROR_CANT_REGISTER_CALLB@ 00011144     sgx_flip_test.obj
 0001:00000168       ??_C@_0BM@COIEDMNF@PVRSRV_ERROR_INVALID_DEVICE?$AA@ 00011168     sgx_flip_test.obj
 0001:00000184       ??_C@_0BH@OEOFFCIM@PVRSRV_ERROR_NOT_OWNER?$AA@ 00011184     sgx_flip_test.obj
 0001:0000019c       ??_C@_0BJ@PHFCJIBD@PVRSRV_ERROR_BAD_MAPPING?$AA@ 0001119c     sgx_flip_test.obj
 0001:000001b8       ??_C@_0BF@KGIMOMJE@PVRSRV_ERROR_TIMEOUT?$AA@ 000111b8     sgx_flip_test.obj
 0001:000001d0       ??_C@_0BI@CDPBDDFH@PVRSRV_ERROR_NO_PRIMARY?$AA@ 000111d0     sgx_flip_test.obj
 0001:000001e8       ??_C@_0BP@FMELGOJO@PVRSRV_ERROR_FLIP_CHAIN_EXISTS?$AA@ 000111e8     sgx_flip_test.obj
 0001:00000208       ??_C@_0BN@JMHJCLJP@ERROR_CANNOT_ACQUIRE_SYSDATA?$AA@ 00011208     sgx_flip_test.obj
 0001:00000228       ??_C@_0BL@JPEIBKNH@PVRSRV_ERROR_SCENE_INVALID?$AA@ 00011228     sgx_flip_test.obj
 0001:00000244       ??_C@_0BK@JAAFMMBM@PVRSRV_ERROR_STREAM_ERROR?$AA@ 00011244     sgx_flip_test.obj
 0001:00000260       ??_C@_0BP@LELIGCIL@PVRSRV_ERROR_INVALID_INTERRUPT?$AA@ 00011260     sgx_flip_test.obj
 0001:00000280       ??_C@_0CB@HFGDLHLE@PVRSRV_ERROR_FAILED_DEPENDENCIES@ 00011280     sgx_flip_test.obj
 0001:000002a4       ??_C@_0BP@PFBLKCEO@PVRSRV_ERROR_CMD_NOT_PROCESSED?$AA@ 000112a4     sgx_flip_test.obj
 0001:000002c4       ??_C@_0BJ@PHLIKBPN@PVRSRV_ERROR_CMD_TOO_BIG?$AA@ 000112c4     sgx_flip_test.obj
 0001:000002e0       ??_C@_0CE@FHHHLEGE@PVRSRV_ERROR_DEVICE_REGISTER_FAI@ 000112e0     sgx_flip_test.obj
 0001:00000304       ??_C@_0BI@JBKNPCOM@PVRSRV_ERROR_FIFO_SPACE?$AA@ 00011304     sgx_flip_test.obj
 0001:0000031c       ??_C@_0BJ@IIGHNIEG@PVRSRV_ERROR_TA_RECOVERY?$AA@ 0001131c     sgx_flip_test.obj
 0001:00000338       ??_C@_0BN@BKNBJNB@PVRSRV_ERROR_INDOSORLOWPOWER?$AA@ 00011338     sgx_flip_test.obj
 0001:00000358       ??_C@_0BM@MCHBLHIP@PVRSRV_ERROR_TOOMANYBUFFERS?$AA@ 00011358     sgx_flip_test.obj
 0001:00000374       ??_C@_0BL@FINKNLDE@PVRSRV_ERROR_NOT_SUPPORTED?$AA@ 00011374     sgx_flip_test.obj
 0001:00000390       ??_C@_0CA@KIDKOOGL@PVRSRV_ERROR_PROCESSING_BLOCKED?$AA@ 00011390     sgx_flip_test.obj
 0001:000003b0       ??_C@_0CA@NBGAMPKE@PVRSRV_ERROR_CANNOT_FLUSH_QUEUE?$AA@ 000113b0     sgx_flip_test.obj
 0001:000003d0       ??_C@_0CE@NLLBGAEA@PVRSRV_ERROR_CANNOT_GET_QUEUE_SP@ 000113d0     sgx_flip_test.obj
 0001:000003f4       ??_C@_0CG@FCILKACH@PVRSRV_ERROR_CANNOT_GET_RENDERDE@ 000113f4     sgx_flip_test.obj
 0001:0000041c       ??_C@_0BD@COEEPPOL@PVRSRV_ERROR_RETRY?$AA@ 0001141c     sgx_flip_test.obj
 0001:00000430       ??_C@_0BJ@IMBALOKG@PVRSRV_DEVICE_ID_UNKNOWN?$AA@ 00011430     sgx_flip_test.obj
 0001:0000044c       ??_C@_0BH@OGEGGGCD@PVRSRV_DEVICE_ID_MSVDX?$AA@ 0001144c     sgx_flip_test.obj
 0001:00000464       ??_C@_0BF@BBCLGMON@PVRSRV_DEVICE_ID_SGX?$AA@ 00011464     sgx_flip_test.obj
 0001:0000047c       ??_C@_0CD@BDGFMHBG@PVRSRV_DEVICE_TYPE_EXT?5?$CI3rd?5Part@ 0001147c     sgx_flip_test.obj
 0001:000004a0       ??_C@_0BE@GEDKFGMC@Not?5recognised?50x?$CFx?$AA@ 000114a0     sgx_flip_test.obj
 0001:000004b4       ??_C@_0BI@ICLDLMDM@?4?4?4?4?5ui32ProcessID?3?$CFlu?6?$AA@ 000114b4     sgx_flip_test.obj
 0001:000004cc       ??_C@_0BD@NOILHFAN@PVRSRVDisconnect?3?6?$AA@ 000114cc     sgx_flip_test.obj
 0001:000004e0       ??_C@_0BH@LMCBNGLN@SGXReleaseClientInfo?3?6?$AA@ 000114e0     sgx_flip_test.obj
 0001:000004f8       ??_C@_0CF@DBFHMBAF@Display?5Class?5API?3?5close?5the?5dev@ 000114f8     sgx_flip_test.obj
 0001:00000520       ??_C@_0CM@LDEJMMMA@Attempt?5to?5destroy?5memory?5contex@ 00011520     sgx_flip_test.obj
 0001:0000054c       ??_C@_0DD@GODBIEMM@Display?5Class?5API?3?5unmap?5display@ 0001154c     sgx_flip_test.obj
 0001:00000580       ??_C@_0EO@CKGGAHCN@Display?5Class?5API?3?5unmap?5swapcha@ 00011580     sgx_flip_test.obj
 0001:000005d0       ??_C@_0CA@OPHIOJCF@ERROR?3?5Flip?5failed?5to?5complete?6?$AA@ 000115d0     sgx_flip_test.obj
 0001:000005f0       ??_C@_0DC@ICDBNIMJ@Surface?5?$CFlu?0?5read?5ops?5complete?3?5@ 000115f0     sgx_flip_test.obj
 0001:00000624       ??_C@_0CC@NAGJIHPE@waiting?5for?5flips?5to?5complete?4?4?4@ 00011624     sgx_flip_test.obj
 0001:00000648       ??_C@_0DE@PBNHKLOP@Display?5Class?5API?3?5ERROR?5unsuppo@ 00011648     sgx_flip_test.obj
 0001:0000067c       ??_C@_0CP@IFAFGPME@Display?5Class?5API?3?5map?5display?5s@ 0001167c     sgx_flip_test.obj
 0001:000006b0       ??_C@_0EK@BPNJOJAB@?4?4?4?4?5Shared?5heap?5?$CFlu?5?9?5HeapID?30x@ 000116b0     sgx_flip_test.obj
 0001:000006fc       ??_C@_0DE@BODOPOHG@Display?5Class?5API?3?5get?5the?5syste@ 000116fc     sgx_flip_test.obj
 0001:00000730       ??_C@_0ED@NNKEOJPF@?4?4?4?4?5Display?5dimensions?5?$CFlu?5?9?5By@ 00011730     sgx_flip_test.obj
 0001:00000774       ??_C@_0DB@DPDHNDGF@Display?5Class?5API?3?5enumerate?5dis@ 00011774     sgx_flip_test.obj
 0001:000007a8       ??_C@_0CK@PAKBMFJN@?4?4?4?4?5Display?5format?5?$CFlu?5?9?5Pixelf@ 000117a8     sgx_flip_test.obj
 0001:000007d4       ??_C@_0O@GDPIEJBG@?4?4?4?4?5Name?3?$CFs?6?$AA@ 000117d4     sgx_flip_test.obj
 0001:000007e4       ??_C@_0BI@BLGHILNJ@?4?4?4?4?5MaxSwapChains?3?$CFlu?6?$AA@ 000117e4     sgx_flip_test.obj
 0001:000007fc       ??_C@_0BO@POAFDAJE@?4?4?4?4?5MaxSwapChainBuffers?3?$CFlu?6?$AA@ 000117fc     sgx_flip_test.obj
 0001:0000081c       ??_C@_0BK@CPCAOBID@?4?4?4?4?5MinSwapInterval?3?$CFlu?6?$AA@ 0001181c     sgx_flip_test.obj
 0001:00000838       ??_C@_0BK@DMGFAHCI@?4?4?4?4?5MaxSwapInterval?3?$CFlu?6?$AA@ 00011838     sgx_flip_test.obj
 0001:00000854       ??_C@_0CO@GIPBIACE@Display?5Class?5API?3?5enumerate?5dis@ 00011854     sgx_flip_test.obj
 0001:00000884       ??_C@_0CF@FMDFFMKC@Display?5Class?5API?3?5Get?5display?5i@ 00011884     sgx_flip_test.obj
 0001:000008ac       ??_C@_0CA@DAONOMAK@Display?5Class?5API?3?5open?5device?6?$AA@ 000118ac     sgx_flip_test.obj
 0001:000008cc       ??_C@_0CL@DNLHEBLI@Attempt?5to?5create?5memory?5context@ 000118cc     sgx_flip_test.obj
 0001:000008f8       ??_C@_0CA@DGGJNKGO@?5Test?5Memory?5Allocation?5FAILED?6?$AA@ 000118f8     sgx_flip_test.obj
 0001:00000918       ??_C@_0DM@CIPNLPOO@PVRSRVEnumerateDeviceClass?$CI?$CJ?5ret@ 00011918     sgx_flip_test.obj
 0001:00000954       ??_C@_0CG@MMBLEMBO@Display?5Class?5API?3?5enumerate?5dev@ 00011954     sgx_flip_test.obj
 0001:0000097c       ??_C@_0BJ@NLALCGOE@Getting?5SGX?5Client?5info?6?$AA@ 0001197c     sgx_flip_test.obj
 0001:00000998       ??_C@_0BP@IDIGABKI@Attempt?5to?5acquire?5device?5?$CFd?3?6?$AA@ 00011998     sgx_flip_test.obj
 0001:000009b8       ??_C@_0BH@PPGIPGOP@?5?5?5?5?5?5?5?5?5?5?5?5?$CF04d?5?5?5?5?$HM?5?$AA@ 000119b8     sgx_flip_test.obj
 0001:000009d0       ??_C@_01EEMJAFIK@?6?$AA@   000119d0     sgx_flip_test.obj
 0001:000009d4       ??_C@_0BK@GEDDINJE@?4?4?4?4?5Reported?5?$CFu?5devices?6?$AA@ 000119d4     sgx_flip_test.obj
 0001:000009f0       ??_C@_0CD@INKLJIDI@?4?4?4?4?5Device?5Number?5?5?$HM?5Device?5Typ@ 000119f0     sgx_flip_test.obj
 0001:00000a14       ??_C@_04LNELOFCG@?5OK?6?$AA@ 00011a14     sgx_flip_test.obj
 0001:00000a1c       ??_C@_0DE@KAFOOJDI@Get?5number?5of?5devices?5from?5PVRSR@ 00011a1c     sgx_flip_test.obj
 0001:00000a50       ??_C@_0M@FBGHFOFL@?5FAIL?5?9?5?$CFs?6?$AA@ 00011a50     sgx_flip_test.obj
 0001:00000a5c       ??_C@_0DH@PPPHAACG@?9?9?9?9?9?9?9?9?9?9?9?9?9?9?9?9?9?9?9?9?9?9?9?5Start?5?9?9@ 00011a5c     sgx_flip_test.obj
 0001:00000a94       ??_C@_0CL@KFFMIBHA@Call?5PVRSRVConnect?5with?5a?5valid?5@ 00011a94     sgx_flip_test.obj
 0001:00000ac0       ??_C@_0DN@ECNCANJG@Swap?5interval?5should?5be?5below?525@ 00011ac0     sgx_flip_test.obj
 0001:00000b00       ??_C@_0DD@CGPFNJKD@Number?5of?5swap?5chain?5buffers?5sho@ 00011b00     sgx_flip_test.obj
 0001:00000b34       ??_C@_02GHOAPKHL@?9b?$AA@  00011b34     sgx_flip_test.obj
 0001:00000b38       ??_C@_02DIMDPHP@?9f?$AA@   00011b38     sgx_flip_test.obj
 0001:00000b40       ??_C@_1KE@BDGMONOJ@?$AAH?$AA?3?$AA?2?$AAW?$AAI?$AAN?$AAC?$AAE?$AA6?$AA0?$AA0?$AA?2?$AAP?$AAL?$AAA?$AAT?$AAF?$AAO?$AAR?$AAM?$AA?2?$AAS?$AAM?$AAD?$AAK?$AAV?$AA2?$AA1?$AA0?$AA?2?$AAS?$AAR@ 00011b40     wince_unittests.obj
 0001:00000be4       ??_C@_1CI@OHCJFJPM@?$AAE?$AAR?$AAR?$AAO?$AAR?$AA?3?$AA?5?$AA?$CF?$AAs?$AA?5?$AAl?$AAi?$AAn?$AAe?$AA?5?$AA?$CF?$AAd?$AA?3?$AA?5?$AA?$AA@ 00011be4     wince_unittests.obj
 0001:00000c0c       ??_C@_1CK@MPGKAOE@?$AA?$CI?$AAe?$AAr?$AAr?$AAo?$AAr?$AA?5?$AAc?$AAo?$AAd?$AAe?$AA?3?$AA?5?$AA?$CF?$AAd?$AA?$CJ?$AA?3?$AA?5?$AA?$CF?$AAs?$AA?$AA@ 00011c0c     wince_unittests.obj
 0001:00000c38       ??_C@_1M@DMCDIEDK@?$AAP?$AAK?$AAM?$AA1?$AA?3?$AA?$AA@ 00011c38     wince_unittests.obj
 0001:00000c44       ??_C@_0L@GPAGIAIC@?9disablepm?$AA@ 00011c44     wince_unittests.obj
 0001:00000c50       ??_C@_07FBLHGNAH@app?4exe?$AA@ 00011c50     wince_unittests.obj
 0001:00000e4c       print_dev_type             00011e4c f   sgx_flip_test.obj
 0001:00000eac       main                       00011eac f   sgx_flip_test.obj
 0001:00001bbc       WinMain                    00012bbc f   wince_unittests.obj
 0001:00001de4       Sleep                      00012de4 f   coredll:COREDLL.dll
 0001:00001df4       ReleasePowerRequirement    00012df4 f   coredll:COREDLL.dll
 0001:00001e04       NKDbgPrintfW               00012e04 f   coredll:COREDLL.dll
 0001:00001e14       FormatMessageW             00012e14 f   coredll:COREDLL.dll
 0001:00001e24       GetLastError               00012e24 f   coredll:COREDLL.dll
 0001:00001e34       SetPowerRequirement        00012e34 f   coredll:COREDLL.dll
 0001:00001e44       WideCharToMultiByte        00012e44 f   coredll:COREDLL.dll
 0001:00001e54       PVRSRVDisconnect           00012e54 f   srvclum:SRVCLUM.dll
 0001:00001e64       SGXReleaseClientInfo       00012e64 f   srvclum:SRVCLUM.dll
 0001:00001e74       PVRSRVCloseDCDevice        00012e74 f   srvclum:SRVCLUM.dll
 0001:00001e84       PVRSRVDestroyDeviceMemContext 00012e84 f   srvclum:SRVCLUM.dll
 0001:00001e94       PVRSRVDestroyDCSwapChain   00012e94 f   srvclum:SRVCLUM.dll
 0001:00001ea4       PVRSRVUnmapDeviceClassMemory 00012ea4 f   srvclum:SRVCLUM.dll
 0001:00001eb4       PVRSRVSwapToDCBuffer       00012eb4 f   srvclum:SRVCLUM.dll
 0001:00001ec4       PVRSRVGetDCBuffers         00012ec4 f   srvclum:SRVCLUM.dll
 0001:00001ed4       PVRSRVCreateDCSwapChain    00012ed4 f   srvclum:SRVCLUM.dll
 0001:00001ee4       PVRSRVMapDeviceClassMemory 00012ee4 f   srvclum:SRVCLUM.dll
 0001:00001ef4       PVRSRVGetDCSystemBuffer    00012ef4 f   srvclum:SRVCLUM.dll
 0001:00001f04       PVRSRVEnumDCDims           00012f04 f   srvclum:SRVCLUM.dll
 0001:00001f14       PVRSRVEnumDCFormats        00012f14 f   srvclum:SRVCLUM.dll
 0001:00001f24       PVRSRVGetDCInfo            00012f24 f   srvclum:SRVCLUM.dll
 0001:00001f34       PVRSRVOpenDCDevice         00012f34 f   srvclum:SRVCLUM.dll
 0001:00001f44       PVRSRVCreateDeviceMemContext 00012f44 f   srvclum:SRVCLUM.dll
 0001:00001f54       PVRSRVEnumerateDeviceClass 00012f54 f   srvclum:SRVCLUM.dll
 0001:00001f64       SGXGetClientInfo           00012f64 f   srvclum:SRVCLUM.dll
 0001:00001f74       PVRSRVAcquireDeviceData    00012f74 f   srvclum:SRVCLUM.dll
 0001:00001f84       PVRSRVEnumerateDevices     00012f84 f   srvclum:SRVCLUM.dll
 0001:00001f94       PVRSRVConnect              00012f94 f   srvclum:SRVCLUM.dll
 0001:00002024       WinMainCRTStartup          00013024 f   corelib0:pegwmain.obj
 0001:00002120       exit                       00013120 f   corelib0:cexit.obj
 0001:00002138       _exit                      00013138 f   corelib0:cexit.obj
 0001:00002178       __GSHandlerCheckCommon     00013178 f   corelib0:gshandler.obj
 0001:000021b4       __GSHandlerCheck           000131b4 f   corelib0:gshandler.obj
 0001:000021d8       __security_init_cookie     000131d8 f   corelib0:seccinit.obj
 0001:00002234       __security_check_cookie    00013234 f   corelib0:armsecgs.obj
 0001:00002248       __gsfailure                00013248 f   corelib0:armsecgs.obj
 0001:0000228c       _initterm                  0001328c f   corelib0:crt0dat.obj
 0001:000022c0       _cinit                     000132c0 f   corelib0:crt0dat.obj
 0001:000022f4       printf                     000132f4 f   corelib1:COREDLL.dll
 0001:00002304       free                       00013304 f   corelib1:COREDLL.dll
 0001:00002314       malloc                     00013314 f   corelib1:COREDLL.dll
 0001:00002324       atol                       00013324 f   corelib1:COREDLL.dll
 0001:00002334       strcmp                     00013334 f   corelib1:COREDLL.dll
 0001:00002344       _stricmp                   00013344 f   corelib1:COREDLL.dll
 0001:00002354       _isctype                   00013354 f   corelib1:COREDLL.dll
 0001:00002364       wcslen                     00013364 f   corelib1:COREDLL.dll
 0001:00002374       memset                     00013374 f   corelib1:COREDLL.dll
 0001:00002384       _XcptFilter                00013384 f   corelib1:COREDLL.dll
 0001:00002394       __C_specific_handler       00013394 f   corelib1:COREDLL.dll
 0001:000023a4       __security_gen_cookie2     000133a4 f   corelib1:COREDLL.dll
 0001:000023b4       __report_gsfailure         000133b4 f   corelib1:COREDLL.dll
 0001:000023c4       TerminateProcess           000133c4 f   coredll:COREDLL.dll
 0001:000023ec       __IMPORT_DESCRIPTOR_COREDLL 000133ec     coredll:COREDLL.dll
 0001:00002400       __IMPORT_DESCRIPTOR_SRVCLUM 00013400     srvclum:SRVCLUM.dll
 0001:00002414       __NULL_IMPORT_DESCRIPTOR   00013414     coredll:COREDLL.dll
 0002:00000000       __imp_Sleep                00014000     coredll:COREDLL.dll
 0002:00000004       __imp_ReleasePowerRequirement 00014004     coredll:COREDLL.dll
 0002:00000008       __imp_NKDbgPrintfW         00014008     coredll:COREDLL.dll
 0002:0000000c       __imp_FormatMessageW       0001400c     coredll:COREDLL.dll
 0002:00000010       __imp_GetLastError         00014010     coredll:COREDLL.dll
 0002:00000014       __imp_SetPowerRequirement  00014014     coredll:COREDLL.dll
 0002:00000018       __imp_WideCharToMultiByte  00014018     coredll:COREDLL.dll
 0002:0000001c       __imp___report_gsfailure   0001401c     corelib1:COREDLL.dll
 0002:00000020       __imp___security_gen_cookie2 00014020     corelib1:COREDLL.dll
 0002:00000024       __imp___C_specific_handler 00014024     corelib1:COREDLL.dll
 0002:00000028       __imp__XcptFilter          00014028     corelib1:COREDLL.dll
 0002:0000002c       __imp_memset               0001402c     corelib1:COREDLL.dll
 0002:00000030       __imp_wcslen               00014030     corelib1:COREDLL.dll
 0002:00000034       __imp__isctype             00014034     corelib1:COREDLL.dll
 0002:00000038       __imp__stricmp             00014038     corelib1:COREDLL.dll
 0002:0000003c       __imp_strcmp               0001403c     corelib1:COREDLL.dll
 0002:00000040       __imp_atol                 00014040     corelib1:COREDLL.dll
 0002:00000044       __imp_malloc               00014044     corelib1:COREDLL.dll
 0002:00000048       __imp_free                 00014048     corelib1:COREDLL.dll
 0002:0000004c       __imp_printf               0001404c     corelib1:COREDLL.dll
 0002:00000050       __imp_TerminateProcess     00014050     coredll:COREDLL.dll
 0002:00000054       \177COREDLL_NULL_THUNK_DATA 00014054     coredll:COREDLL.dll
 0002:00000058       __imp_PVRSRVEnumerateDeviceClass 00014058     srvclum:SRVCLUM.dll
 0002:0000005c       __imp_SGXGetClientInfo     0001405c     srvclum:SRVCLUM.dll
 0002:00000060       __imp_PVRSRVAcquireDeviceData 00014060     srvclum:SRVCLUM.dll
 0002:00000064       __imp_PVRSRVEnumerateDevices 00014064     srvclum:SRVCLUM.dll
 0002:00000068       __imp_PVRSRVConnect        00014068     srvclum:SRVCLUM.dll
 0002:0000006c       __imp_PVRSRVOpenDCDevice   0001406c     srvclum:SRVCLUM.dll
 0002:00000070       __imp_PVRSRVGetDCInfo      00014070     srvclum:SRVCLUM.dll
 0002:00000074       __imp_PVRSRVEnumDCFormats  00014074     srvclum:SRVCLUM.dll
 0002:00000078       __imp_PVRSRVEnumDCDims     00014078     srvclum:SRVCLUM.dll
 0002:0000007c       __imp_PVRSRVGetDCSystemBuffer 0001407c     srvclum:SRVCLUM.dll
 0002:00000080       __imp_PVRSRVMapDeviceClassMemory 00014080     srvclum:SRVCLUM.dll
 0002:00000084       __imp_PVRSRVCreateDCSwapChain 00014084     srvclum:SRVCLUM.dll
 0002:00000088       __imp_PVRSRVGetDCBuffers   00014088     srvclum:SRVCLUM.dll
 0002:0000008c       __imp_PVRSRVSwapToDCBuffer 0001408c     srvclum:SRVCLUM.dll
 0002:00000090       __imp_PVRSRVUnmapDeviceClassMemory 00014090     srvclum:SRVCLUM.dll
 0002:00000094       __imp_PVRSRVDestroyDCSwapChain 00014094     srvclum:SRVCLUM.dll
 0002:00000098       __imp_PVRSRVDestroyDeviceMemContext 00014098     srvclum:SRVCLUM.dll
 0002:0000009c       __imp_PVRSRVCloseDCDevice  0001409c     srvclum:SRVCLUM.dll
 0002:000000a0       __imp_SGXReleaseClientInfo 000140a0     srvclum:SRVCLUM.dll
 0002:000000a4       __imp_PVRSRVDisconnect     000140a4     srvclum:SRVCLUM.dll
 0002:000000a8       __imp_PVRSRVCreateDeviceMemContext 000140a8     srvclum:SRVCLUM.dll
 0002:000000ac       \177SRVCLUM_NULL_THUNK_DATA 000140ac     srvclum:SRVCLUM.dll
 0002:000000b0       __security_cookie          000140b0     corelib0:seccinit.obj
 0002:000000b4       __security_cookie_complement 000140b4     corelib0:seccinit.obj
 0002:000000b8       pfnRegisteredWndProc       000140b8     wince_unittests.obj
 0002:000000bc       _exitflag                  000140bc     corelib0:cexit.obj
 0002:000000c0       __onexitend                000140c0     <common>
 0002:000000c4       __onexitbegin              000140c4     <common>

 entry point at        0001:00002024

 Static symbols

 0001:00000c84       GetString                  00011c84 f   sgx_flip_test.obj
 0001:00001fac       WinMainCRTStartupHelper    00012fac f   corelib0:pegwmain.obj
 0001:00002058       doexit                     00013058 f   corelib0:cexit.obj
